:1000000000308A00DB2800000A108A100A118207DB
:1000100028340C34013406340A108A100A1182077D
:1000200062346C3465343A34253473340A340D3414
:1000300000342F3084008313000803193028013066
:10004000F800BF30F7006400F70B2328F80B2128D5
:100050004A30F700F70B2A2800006400800B1F28A5
:1000600000340708F039B60035080F393604870028
:1000700006148316061064008312061083160610F9
:1000800083120034B308031D4728861048288614BD
:10009000831686108312B40E3408B5003120B40ED6
:1000A0003408B500312064000C30F700F70B5628F7
:1000B000592800341430AF001920F030831687051A
:1000C000831286108316861083120610831606107C
:1000D0008312AB012B08023C031C76280230AF00D0
:1000E00019200330B5003120AB0A6A2864000C30B7
:1000F000F700F70B79287C280230B5003120640026
:100100000C30F700F70B82288528AB012B08023C46
:10011000031C96282B080420AC00B3012C08B40063
:1001200042200230AF001920AB0A86281D29013079
:100130002F02B1003008023C031DA0284030B10757
:1001400031088038B200B3013208B40042200034D4
:100150002E080C3A0319B628063A0319BE28073AA6
:100160000319C428053A0319C928CE28B301013060
:10017000B40042200230AF001920DA280130AF006D
:100180000230B0009720DA280130AF00B00097208D
:10019000DA28B3011030B4004220DA282E081F3CC0
:1001A000031CD4280730AE050130B3002E08B4007C
:1001B0004220DA280034840183131F3083050C3079
:1001C00083169900A6309800903083129800831609
:1001D0001F149F141F159F1107309C00FF308312BE
:1001E000A00083161F149F141F159F1183121F1048
:1001F0008316091283129412A01220088316870016
:10020000831220162008831687008312A01120086D
:10021000831687000030831294008316940001082F
:10022000C73908388100831290010030F80092002D
:1002300000308316920083125A2883160512831207
:1002400005120630AB00FA30AF001920AB0B2329A2
:10025000831605128312051641300C1E2D299900B4
:1002600054300C1E312999000D300C1E352999008F
:100270008C1E38291A08A1008C1E3C291A08A200DD
:10028000A301AB012B080C20AB0AF700AE00A8209D
:1002900004302B02031D42292130840083130030D7
:1002A000000403196329AD010408AC002D10831B61
:1002B0002D140008AE00A8202C08840083132D18EC
:1002C0008317840A4F290A30AE00A8200D30AE00F3
:0602D000A8201D296300B7
:02400E00393F38
:00000001FF
